:100000000C94B9090C94E1090C94E1090C94E109F0
:100010000C94E1090C94E1090C94E1090C94E109B8
:100020000C94E1090C94E1090C9404120C947312E1
:100030000C94E1090C94E1090C94E1090C94E10998
:100040000C94E1090C94E1090C94E1090C94E10988
:100050000C94E1090C94E1090C94E1090C94A514A9
:100060000C94E1090C94E1090C94E1090C94E10968
:100070000C94E1090C94E1090C94E1090C94E10958
:100080000C94E1090C94E1090C94E1090C94E10948
:100090000C94E1090C94E1090C94E1090C94E10938
:1000A0000C94E1090C94E1090C94E1090010400062
:1000B0004040100000000010403000401080000060
:1000C00000104020804010000000000800080008D8
:1000D00000080008000800080008FF0007252900A4
:1000E000062542D04C11300002524AD4095828004B
:1000F000025290900005484200011FF800036A0A6E
:1001000000017F8600032AA803FC018000024A5CEC
:10011000C53E04EFA4000152FB6F070783C700012F
:1001200012474FD2775F34000152C8D52426087693
:10013000000154E29DEA68367200014518EF6D0532
:100140001B3202411ECC21B0B9D652000102BC0DB7
:10015000D812B210000142F96884A424010001C33E
:10016000B8E0EE5052040001BA87545EEB10500024
:100170000154AB1A4EE4444200010837E5D7F94474
:100180000825023A50483490202550644A293C10F2
:100190000249423090405D40484D2817E25FE140FF
:1001A00000014501710CA2A0400469A0121E5EADC1
:1001B00010512A09302EF42850404244398CF52C35
:1001C00000014A5505314A1489504035289C185081
:1001D0003C1092290A3C9539412000014910AF2D6D
:1001E00077A120484A441BF463C29000012A914E33
:1001F000A3C002904462041BE000010A4051420087
:10020000010FF0000102408000020FF00004000224
:100210000FF0000324000207F800011000010100A4
:100220000206DC67A4000188000206F8054100020E
:10023000000203FD4285000122255552AC0003084F
:1002400025000102D86BA000018000020EF04900D9
:100250000300021FE506D80001240002FF00020689
:10026000000101000101FE000201801000010FF0F9
:100270000003604000011FE0000318440001FF007C
:10028000040624F72BCFC29D4C3BFF5AF972AF31C5
:100290007D17F800020AA00002AE1418288A000197
:1002A000AE141822800003AE14182830506A800063
:1002B00005C5909090909095C00001AE141828301C
:1002C0003A800007AE14100005FF00011ABAAAAA6E
:1002D000AA80800001D501D000018055000301D023
:1002E000000180000280D5000501855285528552AB
:1002F0008ABAAAAA8080000255000701D0000180B6
:100300000005FFFFEFF55555BC3CBCBC40FE3C3C36
:10031000BCC6FAAAAAAA3C3CBCBCBC3CC6FAAAAA67
:10032000AAAAAA10109010901095D555BC3CBCBC40
:10033000BCC0FEAAAAAAAAAAAAAA3C3CBFFFFFFF69
:10034000FFFFFF0001153196593C98000118461730
:100350003800025AC32CB2C8A004000118000118CA
:1003600055A4B2CB2CB2C8040A020A020A0A925956
:100370003C9800011800014610CB2CB2CB2CB2C81F
:10038000A400010CA00004FFFFEF95C52B9C181DD5
:100390001C55FF9C101C52E295C52A94181D1C1870
:1003A000183E95C52B8A5715FBF5FDF5FDF5FFC5E4
:1003B000EC98181D1C183DD52B8A5714AE295FB038
:1003C000101FFFFFFFFFFFFF0001155FEABF3E1890
:1003D00014143ABF28180522000135406A841C1401
:1003E000152C387DDFEABFD57FAAAA00051541A0EC
:1003F0000D1C14152C56FABFD57FAAFF55FE1C08FC
:100400001CA00004FFFFE01555418004040455C7FB
:1004100090000255D5400001AA2802000104040002
:10042000015515554000015555FFFFFFFFFFFFEF38
:10043000055185040001040455D5400001555500BF
:1004400001015514800FFFFFFFFFFFF8F9EEBAAA74
:10045000AB3F737F6B6FA86F7F7F80000201A57F2A
:100460007F7F6FFFFF87FAAAAAAAAAAAADF9F9F9B6
:10047000F9F9EF4000017FBF7F6FFFFFAAAAAAAA88
:10048000AAAAAAAAFF7F7F8F9F9F9F9F96698775C1
:10049000FF55F9B8EB13F55533DC07D000020151D5
:1004A000E21A1BFFB43F85D55555555555946990B3
:1004B00069906984400001E75C47F7B47F7F55FF8E
:1004C00055555555528780F9369906990665F4F4C5
:1004D000F1AB52C0800002D50001D400025AFAAA42
:1004E0004AEA220002800001022A94B14FEAAAA43B
:1004F00074F4F4F4F4F4FEFAAA2200028000015429
:10050000D401ABAAAAA52FA80001800F4F4F4F4FCF
:100510004F0520DFFEFF05BC3C3C3C40FE3C3D3C23
:100520003D84855555BC3C3C3C3C3C7DC69534B532
:10053000A4B16520D120D120D5F554BC3C3C3C3C35
:1005400041FFFEE35D4955AA00013C3C33120D1208
:100550000D1205B464F153FA05000118185216384B
:1005600018000170AE0AAAAA1C1819000341054020
:100570005EAA8A2A54B464B464B460FE933C180042
:100580000341D5015471AA962BE2A40001135B46E6
:100590004B464A0692FFFEF800011C181818464206
:1005A0003C081851D55555FF18151D0808082EAAE6
:1005B000AABFF4AA550692F292F292FA0FD5B01899
:1005C0001808085EFFFEFF8A00012BFC6A9C1C17BE
:1005D000292F292F2A6694049155553884100C45EB
:1005E000FB800001103AAAAAAAAABC1414101D107C
:1005F000742A00013546A8AA94940494049405D062
:1006000002883010040220AA0155555554000155A6
:10061000A81415694049404804808FFEFFA5A40234
:10062000020001555582020257D55555FF3C000185
:100630000202000255D555400555FF048080808098
:100640008085407D88000204000155FFFEFFAAAAB4
:10065000AAAAAA2801080808080808025090914A86
:1006600054FF3C7DFF000101FE7F7F00021FEAAACC
:10067000FF7FFFFD3FFF00011FEAAAAAAAAA92502E
:10068000925092509ABA827F7F7F7B7FBF6A0155DA
:1006900055495D55557FFF71250925092202029FA5
:1006A000FE1F01FF5DAC8E8000010303FC52FAA324
:1006B000FAFF551FE2827AB6841555552A80FF024B
:1006C000029202920297D5550002F8F8000195FFB8
:1006D000FEFFAAA2AAFFAAAA8308000129202920B6
:1006E00007FC0E91ABAA2A0001A080D51FC2800092
:1006F000012AFF541A4A800002808000015500013F
:1007000007FA803F9597FC07FC07FC013C54D58015
:100710000001808055D501495D554949000180801F
:10072000897FC07FC07F07909FFEFF05BE3C0CBC49
:10073000416ABC3C3C7D542BA7FF3D3C3C3C3C3CCF
:100740003EAA9784107AFF0790909090909A8C1010
:10075000BC3C3C3C3C5EFFFE23412B0AFFFF3C3C83
:10076000313909090909649262F1A8379A04140021
:100770000141552098104124755752B400011800CA
:1007800001100875D54031451252F492649264927A
:1007900067B14EAC0806040855D501955455525220
:1007A0000001AC180F492649264965909FFEFC3987
:1007B00014940818510001A815145642EAA8FF081D
:1007C00018141C1C1C40FEAA4CF6F8FF6590919072
:1007D00091909A3CBD18181C051C41FFFEC057AAF9
:1007E00007FFFF181805190919091905548491AB59
:1007F000FDBC00011C1C3EAA0404145D52A83F95D8
:1008000094381418141056280001EDD51555945439
:1008100084548454855141B0181414152BAA01AB8B
:1008200040AB4B4A0001BC101155484548440410E8
:100830009FFEE066A4000102000155D5048002324B
:1008400010ABD4FF1C080200010100012A3FD5684B
:100850009341FF04109010901095309F14050200F2
:10086000010455FFFEFF52A603FFFF3C00010901F2
:1008700009010900019512120155F9FFFF7DFF875B
:10088000FAFF7F7D78A80D5154F7FFFF6F7F7F7FC0
:10089000C1FED769BFEA0512151215121AFF6F7F44
:1008A0007F5D7FFF035201AB0B5524250001F77FCD
:1008B000795121512152FAEDFFFEAA0280000280F7
:1008C0002D55000335555AABFF0880021001000179
:1008D0002AAB55000215FFFAEDFAEDFAEDF500012D
:1008E0000B040120000184ADFFFE55F6AADAFFFFDC
:1008F0000800010FAEDFAEDFADFF000510100002F3
:1009000001010008010100060101000910100008A2
:100910000101000DFFFFFFFFFFFFEFFFFFFFFEFFE5
:10092000FFFFFFFFFFFFFFFFFEFFFFFFFFFFFFFFD8
:10093000FEFFFFFFFFFFFFFFFFFFFFEFFFFFFFFFD8
:10094000FFFFFFFFFFFEFFFFFFFFFFFFFFFFFFFFB8
:10095000FFFFFFFFF8F9F9F9F9F9EE1000020101C4
:10096000000107F9FE0004010100060106F9F9F98A
:10097000F9F9F9F9F9F9EE1000057F9FE00101009E
:10098000017F9FE07F9F9F9F9F9F9F9F9F97909139
:100990006990698000050E07F9000E9169906990D1
:1009A000699069906980000509169900020E00019E
:1009B0001F9009169906990699069906679E64F490
:1009C000F4F4F04104A7EA00010804040001041053
:1009D0004157EAAAAAAAAAAAAAAAAA74F4F4F4F401
:1009E000F4F4F4F4F4F0410AAAAAAAA74F4F57EA84
:1009F00002000140400F4F4F4F4F4F4F4F4F4F0797
:100A000090F120D120DFBEFBB700020A01200001D7
:100A1000FFEFBE570009F120D120D120D120D120F5
:100A2000DFBEFAA000020F120D0700010A0001123A
:100A300000010F120D120D120D120D1204A555B466
:100A400064B464F0000144490001040A1400045431
:100A5000492494A94A94A94A9464B464B464B464DB
:100A6000B464B464F01254A94A955B4624490C005E
:100A70000189400F4B464B464B464B464A04A0F279
:100A800092F292F2A9554420000382000155555577
:100A900054202000021011011011F292F292F292F1
:100AA000F292F292F2AA820101101F292F2C280043
:100AB0000220200F292F292F292F292F2A64108463
:100AC000940494000180102AA400020528000280EA
:100AD0008825255552A50248248248D494049404BC
:100AE00094049404940001814A8824824B4940492B
:100AF0000400024A800949404940494049404805AC
:100B000012908080808AAA44000101000302000143
:100B1000A4AA2A2020000348484004019080808035
:100B20008080808080808AA80820A0840908081519
:100B300025000220200908080808080808080805F8
:100B400020925092509081115428000202220001FC
:100B50000919105404A4AA54C255555555825092EF
:100B60005092509250925090854A8A955528250966
:100B7000400400020100010925092509250925096C
:100B80002205148002920295515444810002040807
:100B9000000142448A000180800002101040440499
:100BA00090029202920292029202954D680001A474
:100BB00004090001290544000248200900012920F8
:100BC000292029202920051497FC07FC041910541A
:100BD00024000207FE00011090C0521295254A8998
:100BE0005252509207FC07FC07FC07FC07FC04224A
:100BF000A4A4B125487FC0290900027FC0097FC095
:100C00007FC07FC07FC07F04229290909095418AE0
:100C10000001010003020001A58A941020000320B6
:100C2000000140420290909090909090909090950A
:100C300008400001AC28010909082000040909093D
:100C4000090909090909096120F4926492605410A4
:100C500054A400020A4A00022001480954AA548AF6
:100C6000951548AA74926492649264926492604169
:100C7000555450A52E492651050002A4900F49262F
:100C8000492649264926496514859091909B74B25E
:100C9000100001AAAAAA0001AA96C96552A00005DF
:100CA00040510001919091909190919091909B2D45
:100CB000941164240919090524AAAAA00AA31909F0
:100CC000190919091909190492145484548925B26F
:100CD000454ADFD55524F526C96C8485255292AA4C
:100CE0005252542294548454845484548454892CED
:100CF000924ABD494045484889DD55524F505548B4
:100D00004548454845484402A290109010992D92BC
:100D1000101441000105000155825B2C2410941031
:100D20000002844040881010901090109010901095
:100D30009965B40001043449410908441100015087
:100D40000558410901090109010900019608051228
:100D500015121B6C965491BFAAA925AF10DB653202
:100D600094D12A5492A11554420512151215121548
:100D70001215121B25B552B5651151212A35BFAA8E
:100D8000892BA85121512151215121521552105026
:100D9000105000010223113D0C65216044444400C1
:100DA0000144262C29022264444212105010501093
:100DB000501050105000012412122CB6D1450101E0
:100DC0002D6C442230424401050105010501043126
:100DD0000142553225252868227515110515151172
:100DE0002251509155532A2A9112533282252215AD
:100DF0003225221532252535305551409221535048
:100E0000D55511109110525221532252215321EDE8
:100E1000DD8CC8CCC8C8C585CCE0CCCDD9D8CCCC6D
:100E2000CC8CCC4C208CC5C44CCC8CCC5CC8CCC8F5
:100E3000CCC8CCC8CCC8C8CCCD8921D2DECC8C8D56
:100E4000E1CCCCCC5CDD8C8CCC8CCC8CCC8CCC999F
:100E5000111110111110101010F989111010110832
:100E600019011111B989111101110001111111118B
:100E70001011111110111110111101BA699991017C
:100E800001F9991101011108191101111111011034
:100E900099999889898889898989019899999989DD
:100EA0009199989888000198998998989999989813
:100EB00088898988888989888989899910000108A1
:100EC000889899118888989899919988989888888D
:100ED000989932233332333332323232332332224F
:100EE0003233223323333333233233233322332336
:100EF00033333233333332333332333223333333D6
:100F00003323223333332323322233332333333314
:100F100023320040004000000000000000000100FB
:100F2000000101000080BF00000442020200010134
:100F300000002442000021430001000101000000E4
:100F400000000020C14E6F20616E696D6174696F91
:100F50006E732E20417761697420666F7220302E87
:100F6000302E350000010000FFD5F08D14A1C8819E
:100F7000CFD9F1AF2000F0F89C8E8783878E9CF844
:100F8000F00000FEFF0303030303070EFCF800005C
:100F9000FEFF0303030303070EFCF80000FFFF003E
:100FA000000000000000FFFF0000FEFF838383833A
:100FB00083C7EE7C380000F8FC0E07030303070E1E
:100FC000FCF800003F7FE0C08080C0E07F3FFFFF73
:100FD00001010101010101FFFF0000FFFF0C0C0CEA
:100FE0000C1C3E77E3C100007FFFC0C0C0C0C0E062
:100FF000703F1F00001F3F70E0C0C0C0E0703F1F87
:1010000000007FFFC1C1C1C1C1E3773E1C00001FCA
:101010003F70E0C0C0C0E0703F1F00000000000152
:10102000FFFF010000000008D000000234004083F0
:101030000C0001F90040003E0008C9011000270023
:1010400004000A000100001000270004000A00014B
:1010500000000F00270004000A000100000000004B
:1010600000000000040404040400040A0A0A00004A
:1010700000000A1F0A1F0A0A0A040E140C0A1C08A0
:101080001A1A04040A1A1A0C12140814120C040472
:101090000400000000020408080804020804020218
:1010A00002040800150E1F0E15000004041F04049E
:1010B00000000000000004080000001F0000000005
:1010C000000000000004010204081010100E1113AB
:1010D0001519110E040C040404040E1E110102045F
:1010E000081F1E11010E01111E02060A121F020224
:1010F0001F101E0101111E0E10101E11110E1F01D6
:1011000002040808080E11110E11110E0E11110F14
:1011100001010E00040000000400000400000004AF
:10112000080204081008040200001F001F00000845
:101130000402010204080E1101020400040E11173A
:101140001515190E0E11111F1111111E11111E115D
:10115000111E0E11101010110E1C12111111121C63
:101160001F10101E10101F1F10101E1010100E1137
:10117000101711110F1111111F1111110E04040478
:1011800004040E0101010101110E111214181412B0
:10119000111010101010101F111B15151111111125
:1011A0001915131111110E11111111110E1E11111A
:1011B0001E1010100E11111111120D1E11111E14FE
:1011C00012110F10100E01011E1F04040404040468
:1011D0001111111111110E11111111110A04111116
:1011E0001115151B1111110A040A111111110A040C
:1011F0000404041F01020408101F0E080808080850
:101200000E100804020101010E02020202020E0485
:101210000A11000000000000000000001F08040286
:101220000000000000000E010F110F10101E111120
:10123000111E00000E1010100E01010F1111110FE0
:1012400000000E111F100E0204040E04040400001E
:101250000F11110F0110101E1111111104000C04B7
:1012600004040E02000202020212101012141814DA
:10127000120C04040404040E00001A1515151500C0
:10128000001E1111111100000E1111110E00001E8F
:1012900011111E1000000F11110F0100000E11108E
:1012A000101000000F100E011E04040E04040402AE
:1012B0000000111111110E00001111110A0400009B
:1012C000111115150A0000110A040A11000011116C
:1012D0000F010E00001F0204081F0204040804048A
:1012E00002040404040404040804040204040808B6
:1012F00015020000000001020304050607080900AA
:101300000A0000080B0002020200000904000001AC
:10131000020200000524001001052401010104243B
:101320000206052406000107058103100040090498
:101330000100020A00000007050202400000070544
:1013400083024000000403090412010002EF0201BD
:101350004041233680000101020301417264756936
:101360006E6F204C4C430041726475626F790000CF
:10137000221511241FBECFEFDAE0DEBFCDBF11E092
:10138000A0E0B1E0EAE8FEE302C005900D92AA33C6
:10139000B107D9F728E0AAE3B1E001C01D92A73157
:1013A000B207E1F719E0C9EBD9E004C02197FE01CB
:1013B0000E942E1FC83BD107C9F70E9437150C9415
:1013C000431F0C940000E7E1F4E0A0E0B8E00080E7
:1013D0000EBC8111012C1197A0FDFDCF0192B9F730
:1013E0000DB40895FC0180911604882311F13FB7D4
:1013F000F89482E08093E9002091F200822F90E03F
:101400001816190614F481E090E0882339F0289822
:1014100044E6409315044091F1004083222339F0C3
:101420002091F200211103C02BE62093E8003FBF7A
:1014300008958FEF9FEF08952FB7F89483E080937E
:10144000E9009091E800892F807295FF04C0909187
:10145000F20080E4891B2FBF089580910D04811153
:101460000DC082E08093090484E080930A04109206
:101470000C0410920B0481E080930D0489E094E049
:101480000895CF93DF931F92CDB7DEB76983DC0158
:10149000ED91FC910280F381E02D41E050E0BE012E
:1014A0006F5F7F4F09950F90DF91CF91089583E093
:1014B0008093E9008091F200882319F08AE38093F9
:1014C000E80008950E941C0A90E00895CF93DF93EE
:1014D0001F92CDB7DEB7FC018485958597FD08C0C6
:1014E0002FEF3FEF358724870F90DF91CF9108953D
:1014F000CE0101960E94F209019719F4898190E0CA
:10150000F3CF8FEF9FEFF0CF0F931F93CF93DF9326
:101510001F92CDB7DEB78C01FC018485958597FFBE
:101520000BC0CE0101960E94F209019771F48981E6
:1015300090E0F80195878487F801848595850F9060
:10154000DF91CF911F910F9108958FEF9FEFF1CF12
:10155000FC018485958597FD0BC09FB7F89482E0C8
:101560008093E9008091F2009FBF90E0019608957A
:101570009FB7F89482E08093E9008091F2009FBFCA
:1015800090E008954091B3035091B4032091B103CA
:101590003091B20342175307B4F49091E80095706C
:1015A000E1F39091E80092FD19C08093F1008091E1
:1015B000B3039091B40301968F739927892B19F483
:1015C0008EEF8093E8008091B3039091B40301966D
:1015D0009093B4038093B30381E0089580E008956D
:1015E000DF92EF92FF920F931F93CF93DF93D82E4A
:1015F0008A01EB017B01E40EF51ECE15DF0559F0E3
:10160000D7FE12C0FE0184910E94C20A2196811168
:10161000F4CF0FEF1FEFC801DF91CF911F910F9112
:10162000FF90EF90DF9008958881EECF0F931F9386
:10163000CF93DF931F92CDB7DEB782E0898342E478
:1016400050E063E073E180E80E94F00A0E942D0AF6
:10165000DC0112960D911C910115110589F0D8013C
:10166000ED91FC910280F381E02DBE016F5F7F4F11
:10167000C801099597FD04C0F80100851185ECCFDC
:1016800089810F90DF91CF911F910F910895615043
:1016900030F02091F100FC0120830196F8CF2898CA
:1016A00084E6809315040895FC010E94EB0B3197AA
:1016B00028F068517C4F8F4F9F4FF9CFAB01FC0151
:1016C0000E94EB0B641775078E079F07C8F30895F8
:1016D0008F929F92AF92BF92CF92DF92EF92FF9242
:1016E0000F931F93CF93DF936C017B018A0180914D
:1016F0000F01882309F45AC080911604882309F445
:1017000055C08091B80380FF05C08091E0008260E1
:101710008093E000E801B12C8AEFA82E93E0892E97
:101720002AE3922E209711F4BB20C9F10E941C0AD3
:10173000811108C0AA94AA20C9F181E090E00E941A
:10174000540BF0CF8C171D0611F00CF08C2F9FB7A7
:10175000F8948092E9002091E80025FD02C09FBF27
:10176000E1CF282F30E0C21BD30BF701815020F0CE
:1017700041914093F100FACFE20EF31EBB2021F01D
:101780009092E800B12CEBCF8091E80085FDE7CF87
:101790009092E800BB24B394209709F3F3CF5D98AF
:1017A00084E68093B703101611063CF081E090E0C8
:1017B000F6019383828310E000E0C801DF91CF91AE
:1017C0001F910F91FF90EF90DF90CF90BF90AF905F
:1017D0009F908F900895ADEAB3E02FB7F8947D9174
:1017E0008D919C9166B52FBFA89B05C06F3F18F4E3
:1017F0007F5F8F4F9F4F22E0660F771F881F991FD3
:101800002A95D1F7089590E00C94540B8FB18095F0
:10181000807F669B88601C9B84600895CF93C82F4F
:101820000E94060C982F9C2381E09C1380E0CF91AE
:1018300008952F923F924F925F926F927F928F9274
:101840009F92AF92BF92CF92DF92EF92FF920F934F
:101850001F93CF93DF93CDB7DEB72A970FB6F894D7
:10186000DEBF0FBECDBF25E4289FF001299FF00DFC
:101870001124E35FFC4F21E021831482138216823E
:10188000158228E33FE0009739F02EE13FE08130F8
:10189000910511F030E020E045E4489FF001499FB8
:1018A000F00D1124E35FFC4F4281842E912C8901BD
:1018B0000B5F1F4FA901475F5F4F5A874987B901E7
:1018C0006F5F7F4F50E040E0DF011396BA83A9833A
:1018D000DC01A05FBE4FBE83AD83DC01A45EBE4FC2
:1018E000B887AF8380E1682E712C481559050CF03C
:1018F0009AC04032510509F496C0F9013496E4913A
:101900008E2F90E09C838B83F12CE12CAB81BC81EA
:10191000EA16FB060CF079C0A981BA81AD90BC90A3
:10192000AD81BE818C918A151B0409F00CF46DC049
:10193000AF81B885EC91C5010196A981BA818D93DB
:101940009C93AE0EB11CE4E1EA9DD001EB9DB00D7D
:101950001124AF5CBD4F52964C935297F90184917C
:1019600051968C935197FB01849150968C9350978C
:10197000853008F041C0FBE08F02C0011124FC015A
:10198000EA5DFF4EC590D4901D96DC92CE921C97D6
:10199000FC01E85DFF4EC590D4901F96DC92CE927C
:1019A0001E97F801259035904590549084E18A9DCA
:1019B000D0018B9DB00D1124AF5CBD4F2D923D9297
:1019C0004D925C921397E985FA85A590B590C590E4
:1019D000D4901496AD92BD92CD92DC921797189642
:1019E000AD92BD92CD92DC921B9791E053969C9361
:1019F000AFEFEA1AFA0A8ACF1D967C926E921C9774
:101A00001F967C926E921E97CCCF4F5F5F4F235FE5
:101A10003F4F035F1F4F89859A850D969A87898767
:101A2000635F7F4F62CF2A960FB6F894DEBF0FBE7A
:101A3000CDBFDF91CF911F910F91FF90EF90DF907D
:101A4000CF90BF90AF909F908F907F906F905F905E
:101A50004F903F902F90089525E4289FF001299FF3
:101A6000F00D1124E35FFC4F1082118221E00097FA
:101A700029F022E08130910509F020E035E4389F1B
:101A8000F001399FF00D1124E35FFC4F2283148293
:101A9000138216821582148A138A009749F10197DE
:101AA000E9F0F0E0E0E090E080E0E491EE23D9F0AE
:101AB000FC0185919591A591B491582F492F3A2F0A
:101AC0002B2F852F942FA32FB22F80933A01909321
:101AD0003B01A0933C01B0933D010895E4E6FFE093
:101AE00086E19FE0E2CF50E040E030E020E0E9CF47
:101AF000E5E6FFE08AE19FE0D8CF009731F0EEE124
:101B0000FFE0019721F080E00895E8E3FFE0DB01CA
:101B100052968C9187FDF7CFBDE08B02E00DF11D51
:101B200011243296849108952F923F924F925F92A2
:101B30006F927F928F929F92AF92BF92CF92DF92DD
:101B4000EF92FF920F931F93CF93DF93CDB7DEB742
:101B5000C254D1090FB6F894DEBF0FBECDBF219697
:101B60009FAF8EAF219723967FAF6EAF23975CAF69
:101B70004BAF20910201309103013AAF29AF312CD4
:101B8000212C25E449AD5AAD249FC001259F900D1D
:101B90001124FC01E05FFC4FFEABEDAB445E5E4FF9
:101BA00058AF4FAB23962EAD3FAD23972216330689
:101BB0000CF0FBC32196EEADFFAD2197E20DF31DB6
:101BC000E491EB3070F5F0E0E851F24F0C942E1FE9
:101BD000F30D150E590E9F0EE50E2B0F710FB70F5B
:101BE000FD0F43106F1080919F03811104C08091FD
:101BF000A0038823B1F081E090E0909303018093EB
:101C0000020180915303811104C081E090E00E94A1
:101C1000190C109252031092270210922602109271
:101C20003002FFEF2F1A3F0ABDCF8091A303882314
:101C3000C1F3EDA9FEA9C080D180F12CE12CB4E163
:101C4000BB2EEC14FD046CF7EFA9F8AD80818E0D6E
:101C50009F2D911DB89E8001B99E100D11240F5C1F
:101C60001D4FF8018389882301F181898230E9F4CD
:101C700020E030E0A90160817181828193810E941E
:101C8000631DF801608371838283938320E030E0D9
:101C900040E850E464817581868197810E94621DCD
:101CA000F8016483758386839783FFEFEF1AFF0A39
:101CB000C8CF8091A403882309F4B3CFEDA9FEA96E
:101CC000C080D180F12CE12CA4E1BA2EEC14FD04EB
:101CD0000CF0A7CFEFA9F8AD80818E0D9F2D911D3F
:101CE000B89E8001B99E100D11240F5C1D4FF801A4
:101CF0008389882301F181898230E9F420E030E092
:101D0000A90160817181828193810E94631DF80124
:101D1000608371838283938320E030E040E850E465
:101D200064817581868197810E94631DF8016483B7
:101D3000758386839783FFEFEF1AFF0AC7CF8091E1
:101D4000A103882309F46DCFEDA9FEA9C080D1803D
:101D5000F12CE12CF4E1BF2EEC14FD040CF061CF6A
:101D6000EFA9F8AD80818E0D9F2D911DB89E800149
:101D7000B99E100D11240F5C1D4FF8018389882333
:101D800001F181898230E9F420E030E040E850E45C
:101D900060817181828193810E94621DF80160835C
:101DA00071838283938320E030E0A901648175818F
:101DB000868197810E94631DF80164837583868301
:101DC0009783FFEFEF1AFF0AC7CF8091A203882302
:101DD00009F427CFEDA9FEA9C080D180F12CE12C18
:101DE000E4E1BE2EEC14FD040CF01BCFEFA9F8AD1E
:101DF00080818E0D9F2D911DB89E8001B99E100D82
:101E000011240F5C1D4FF8018389882301F181891A
:101E10008230E9F420E030E040E850E460817181F4
:101E2000828193810E94631DF801608371838283A4
:101E3000938320E030E0A9016481758186819781D8
:101E40000E94631DF8016483758386839783FFEF87
:101E5000EF1AFF0AC7CF8091A303882309F4E1CECC
:101E6000EDA9FEA9C080D180F12CE12C74E1B72E40
:101E7000EC14FD040CF0D5CEEFA9F8AD80818E0DE9
:101E80009F2D911DB89E8001B99E100D11240F5CED
:101E90001D4FF8018389882301F181898230E9F49B
:101EA00020E030E0A90160817181828193810E94EC
:101EB000631DF801608371838283938320E030E0A7
:101EC00040E850E464817581868197810E94621D9B
:101ED000F8016483758386839783FFEFEF1AFF0A07
:101EE000C7CF8091A403882309F49BCEEDA9FEA956
:101EF000C080D180F12CE12C64E1B62EEC14FD04FD
:101F00000CF08FCEEFA9F8AD80818E0D9F2D911D25
:101F1000B89E8001B99E100D11240F5C1D4FF80171
:101F20008389882301F181898230E9F420E030E05F
:101F3000A90160817181828193810E94631DF801F2
:101F4000608371838283938320E030E040E850E433
:101F500064817581868197810E94631DF801648385
:101F6000758386839783FFEFEF1AFF0AC7CF8091AF
:101F7000A103882309F455CEEDA9FEA9C080D18024
:101F8000F12CE12C54E1B52EEC14FD040CF049CEFB
:101F9000EFA9F8AD80818E0D9F2D911DB89E800117
:101FA000B99E100D11240F5C1D4FF8018389882301
:101FB00001F181898230E9F420E030E040E850E42A
:101FC00060817181828193810E94621DF80160832A
:101FD00071838283938320E030E0A901648175815D
:101FE000868197810E94631DF801648375838683CF
:101FF0009783FFEFEF1AFF0AC7CF8091A2038823D0
:1020000009F40FCEEDA9FEA9C080D180F12CE12CFE
:1020100044E1B42EEC14FD040CF003CEEFA9F8ADAE
:1020200080818E0D9F2D911DB89E8001B99E100D4F
:1020300011240F5C1D4FF8018389882301F18189E8
:102040008230E9F420E030E040E850E460817181C2
:10205000828193810E94631DF80160837183828372
:10206000938320E030E0A9016481758186819781A6
:102070000E94631DF8016483758386839783FFEF55
:10208000EF1AFF0AC7CF2BAD3CAD2130310509F067
:10209000C8CDEDA9FEA92081318190E080E064E106
:1020A000821793070CF0BDCDEFA9F8AD4081480F22
:1020B000592F511D649FF001659FF00D1124EF5CB5
:1020C000FD4F4389442349F04189423031F48093E4
:1020D000010181E080933002A4CD0196E1CF2BADC8
:1020E0003CAD232B09F09DCDE6E6FFE02591349130
:1020F000E8E6FFE0849187FF34C037FD26C1232B3B
:1021000009F023C1DE01119610E000E0F801EB5B5D
:10211000F04F8491882339F0E4910F5F1F4FED93C6
:102120000F31110599F7E1E0F0E0EC0FFD1FE00F32
:10213000F11F1082809126029091270242E451E023
:1021400030E020E0281739070CF002C14A5D5F4FEC
:10215000FA01B6976081662309F408C12F5F3F4FEB
:10216000F1CF49AD5AAD4115510509F4BDC041301B
:10217000510509F4E7C0812C912C5401CE018196C0
:102180006C01C501B4010E94D41D2B013C01411416
:1021900051046104710409F4A1C08E010F5F1F4F47
:1021A000F12CE12C16161706180619060CF481C03E
:1021B000F60187010115110509F070C0EC0CFD1C3A
:1021C000C301B2010E940C1E9B01AC01C501B40108
:1021D0000E94621D2B013C012FE632E143E05AE3ED
:1021E0000E94BC1E87FF1BC0F7011082DE01919682
:1021F000FE0131968D91882309F495CF0F31110599
:1022000009F491CF81930F5F1F4FF4CF812C912C54
:102210005401FE01B1966F01B4CF7601E5CF8EE295
:10222000F70180836701F4E0CF0ED11C97012F5F87
:102230003F4F790120E030E040E251E4C301B201B8
:102240000E94C11E2B013C010E94D41D4B017EAF98
:102250006DAF072E000C880B990B0E940C1E9B0182
:10226000AC01C301B2010E94621D2B013C0181142B
:10227000910459F0C701019620E3280DF70120834E
:10228000C816D90651F27C01D5CF2DEC3CEC4CE4BC
:102290005DE30E94CF1D87FFEDCFA6CF015011094E
:1022A000A1E0B0E0AC0FBD1FA00FB11F8C918193D6
:1022B00081CFFBE0EF16F10409F47ACF2FEFE21A99
:1022C000F20A2AE030E040E050E00E94211D605D0B
:1022D000F80161938F01B901CA0164CF80E389835A
:1022E000EE24E394F12C64CFE5E6FFE0082E000C29
:1022F000990BE80FF91FE491EE2309F487CF880FBB
:10230000991F880F991FFC01E65CFE4F8080918029
:10231000A280B38020E030E0A901C501B4010E9491
:10232000CF1DAE014F5D5F4F6A0187FF2ACF8DE25F
:1023300089A3B7FAB094B7F8B0949E012E5D3F4FD1
:1023400069011FCFE4E6FFE0D1CF10E000E0EBCE63
:102350008630910509F465CC9C012F5F3F4F309387
:1023600027022093260297FD5CCC9C0146E2429F07
:10237000C001439F900D11248C010E5B1E4FF8018C
:1023800010822AE030E0328321833483238321E0EA
:1023900025834FE150E0BE016F5F7F4F885B9E4F0A
:1023A0000E94341FF80115A23CCCCE5BDF4F0FB664
:1023B000F894DEBF0FBECDBFDF91CF911F910F917B
:1023C000FF90EF90DF90CF90BF90AF909F908F9055
:1023D0007F906F905F904F903F902F900895AB014A
:1023E00061E08230910508F060E070E0009729F02C
:1023F000019739F090E080E002C082E093E10C9414
:10240000940D80E093E1FBCF1F920F920FB60F92D5
:1024100011248F939F938091E1009091E100937F2D
:102420009093E10083FF0FC01092E90091E0909338
:10243000EB001092EC0092E39093ED0010921604E2
:1024400098E09093F00082FF22C093E09093E9001F
:102450009091F200992319F09AE39093E8009091FB
:10246000B703992341F09091B70391509093B7032C
:10247000911101C05D9A90911504992341F09091BA
:102480001504915090931504911101C0289A84FF6E
:1024900018C08091E2008E7E81608093E20080917E
:1024A000E1008F7E8093E1008091B8038E7E806191
:1024B0008093B8039F918F910F900FBE0F901F9044
:1024C000189580FFF7CF8091E2008E7E8061809327
:1024D000E2008091E1008E7E8093E1008091B8035C
:1024E0008E7E8160E5CF1F920F920FB60F9211245E
:1024F000CF92DF92EF92FF920F931F932F933F9310
:102500004F935F936F937F938F939F93AF93BF93FB
:10251000EF93FF93CF93DF93CDB7DEB76C97DEBF1A
:10252000CDBF1092E9008091E80083FF25C068E0EC
:10253000CE0145960E94470B82EF8093E8008D897B
:1025400087FF39C09091E80090FFFCCF982F9076DC
:1025500009F034C19E894F89588D2F89F88C9111CB
:1025600031C0803861F58091B6038093F1001092FC
:10257000F1008EEF8093E8006C960FB6F894DEBF02
:102580000FBECDBFDF91CF91FF91EF91BF91AF9182
:102590009F918F917F916F915F914F913F912F917B
:1025A0001F910F91FF90EF90DF90CF900F900FBE93
:1025B0000F901F9018959EEF9093E800C7CF109250
:1025C000F100D5CF913059F48111D3CF413051056D
:1025D00081F68091B6038D7F8093B603CACF933086
:1025E00049F48111C6CF4130510519F68091B603E7
:1025F0008260F2CF953041F48091E80080FFFCCFFB
:1026000020682093E300B5CF963009F0A9C00B8D68
:102610001C8D22E01092E9001092B4031092B303D3
:10262000F2122EC01092B2031092B1030E94160B48
:102630001F8299E09983FA8291E09E8390EA9887BD
:102640009AEF99872091B3033091B403275F3F4FEE
:102650003C832B838D831092E9001092B403109277
:10266000B3031093B2030093B10349E050E0BE01FD
:102670006F5F7F4F80E00E94F00A0E94160B79CFB7
:102680001093B2030093B1030E942D0ADC0112964D
:102690000D911C910115110509F451C1D801ED915D
:1026A000FC910480F581E02DBE016B5E7F4FC80177
:1026B0000995009709F03EC1F80100851185EACF20
:1026C000F3E0FF120EC08F89882309F440C08230E6
:1026D00061F440E867E087E693E10E94EF1481111E
:1026E00048CF81E28093EB0047CF813029F440E866
:1026F0006BE08BE593E1F1CF833099F70E942D0ACF
:10270000DC011296ED90FC908E010F5F1F4F680167
:10271000E114F10479F0D701ED91FC910680F78185
:10272000E02DB801C7010995080F111DF701E084DC
:10273000F184EECFD8011C92F60101900020E9F758
:102740003197BF016C197D0940E0C601C6CF65E431
:1027500073E1FB01449150E080E80E94F00A09CF48
:10276000973009F4BECF983021F481E08093F100D6
:1027700000CF993009F0FDCE837009F0B2CFE1E2CD
:10278000F1E081E031E096E32191222371F0809322
:10279000E9003093EB00DF0111972C912093EC00BE
:1027A0009093ED008F5F873079F78EE78093EA0092
:1027B0001092EA008F8980931604DBCE8B8D9C8D5E
:1027C0001092E9001092B4031092B3039093B203F5
:1027D0008093B103898D811192C08E899D89913A30
:1027E00049F4813209F07DCF47E050E068E071E0C4
:1027F00080E0B3CF913209F074CF833269F48F89CE
:10280000988DB0E0A0E08093040190930501A0931F
:102810000601B0930701ADCE803269F48091E800E3
:1028200082FFFCCF67E088E091E00E94470B8BEFCE
:102830008093E8009ECE823209F09BCE8F898093F0
:102840000F01EEEFFFE7859194918B3F9C4D51F185
:10285000E0E0F8E08091080190910901A0910A015F
:10286000B0910B01803B9440A105B105F1F480913A
:102870000F0180FD1AC0EE3F8AE0F80789F587E76F
:1028800097E791838083809160008093B50388E10E
:102890009BE00FB6F894A895809360000FBE9093CC
:1028A000600067CEEEEFFAE0D5CF80819181873767
:1028B000974709F05ECEA89580916000886180936B
:1028C00060008091B50380936000EE3F2AE0F2073C
:1028D00089F08091FE0A9091FF0A9183808349CE0E
:1028E000808191818737980751F29093FF0A8093F6
:1028F000FE0AC5CF1092FF0A1092FE0A3ACE0E943D
:102900002D0ADC0112960D911C910115110509F497
:10291000E8CED801ED91FC910190F081E02DBE014F
:102920006B5E7F4FC8010995811123CEF8010085A8
:102930001185EBCF181619060CF41BCED2CEF1E0A0
:10294000FF12BECE69E473E104CF0F920FB68F93EE
:102950009F93EF93FF938091A8038D5F8D3708F0CD
:102960008D578093A803E9EAF3E080818E4F80833E
:1029700091819F4F918382818F4F828383818F4F7B
:102980008383EDEAF3E080818F5F808381818F4FC5
:10299000818382818F4F828383818F4F83838FB125
:1029A0008F6066991C9B88278F3681F48091A703DE
:1029B000981B963068F0E0E0F8E087E78083818339
:1029C00088E180936000F0936000FFCF9093A703AD
:1029D000FF91EF919F918F910FBE0F901895EF92FD
:1029E000FF920F931F93CF93DF93F82E192FE62EAC
:1029F000042F81E0860F880F0E94C20A83E00E94A4
:102A0000C20ACF2DD12FEC0EFD2EF11CCE15DF0505
:102A1000B9F007FF13C0FE0184910E94C20A182F6B
:102A200080E00E94C20A812321968111EFCFDF91BD
:102A3000CF911F910F91FF90EF9008958881EDCF76
:102A400081E0F5CFE9EBF3E01382128288EE93E0A8
:102A5000A0E0B0E084839583A683B7838BE291E006
:102A6000918380838FEF9FEF958784870895CDB7FB
:102A7000DEB7C856D109DEBFCDBF789483E084BDF0
:102A800083E085BD81E080936E00E1E8F0E083E0C3
:102A90008083E0E881E08083E1E983E08083E0E90E
:102AA00081E08083E1EC87E08083E3EC81E0808358
:102AB000E0EC82E08083E2EC81E08083EAE787E07B
:102AC000808380688083109216041092B60310925F
:102AD000B8038091D70081608093D70080EA80930B
:102AE000D80089B5806189BD89B5826089BD09B486
:102AF00000FEFDCF81E090E00E94540B8091D80051
:102B00008F7C80618093D8008091E000807F8093EB
:102B1000E0008091E1008E7E8093E1008DE0809363
:102B2000E200559A209A81EC80937C0081EF85B970
:102B300087EE84B982E38BB982EF8AB9769A6E9870
:102B400080EF81BB10BA80E58CBD81E08DBD85E052
:102B50000E94030C5F9A85E00E94030C5C98E9E6F2
:102B6000FFE085918EBD00000DB407FEFDCFE63776
:102B7000C1F75C9A81E88093640081E080936500EE
:102B800080E00E94E30980E80E940E0C8823A9F0EF
:102B90005C9885EA8EBD00000DB407FEFDCF5C9AFF
:102BA0002E982F982D988091640080628093640005
:102BB00081E083BF889513BEFCCF84E00E940E0C99
:102BC0008823B9F12D9884E80E940E0C8823A1F087
:102BD0002D9A88EC0E94030C2F986FEF82E090E012
:102BE0000E940F1D84EF91E00E94540B2F9A84E8FD
:102BF0000E940E0C8111FBCF84E10E940E0C8823F1
:102C0000A1F02D9A88EC0E94030C2E9860E082E0DF
:102C100090E00E940F1D84EF91E00E94540B2E9AC9
:102C200084E10E940E0C8111FBCF88EC0E94030C02
:102C3000C4CF2D9A82E090E00E94071D882309F4FA
:102C40005CC03E9A3F9A81E090E00E94071D282FC9
:102C50002470D22E81FF0CC021112E9801EF1FEF9E
:102C600080E40E940E0C882309F44AC02E9A2F9A01
:102C700082E30E94030C0E94060C8111F9CF80E1CF
:102C80008093000190E080E00E942C0D81E090E0B4
:102C90000E942C0D109203011092020190E080E03E
:102CA0000E942C0D90E080E00E94190C80E890E0DA
:102CB00090939A038093990388E790E09093980308
:102CC00080939703BE016F5F7F4F23967FAF6EAFF8
:102CD0002397CE01079625969FAF8EAF25978091BB
:102CE0004001882309F47DC01092400180E090E00B
:102CF000892BA9F30E940000F2CF3E983F98A3CF02
:102D0000DD2029F00430110511F42E9A2F9881E06E
:102D10000E94E309302F3770C32E9801B3E0359538
:102D20002795BA95E1F7C9019695982F8827979529
:102D30008795895E9B4FF12CE12C2E3F4FEF340796
:102D400071F1BC016C567F4FDC0150E040E0F701AF
:102D5000EA58F04F5F01F501E40FF51FE491F0E050
:102D60003F010C2C02C0660C771C0A94E2F72F3F3F
:102D7000320739F054969C905497962854969C921A
:102D80005497CC2021F0FB019080972890824F5FD0
:102D90005F4F6F5F7F4F119648355105E1F62F5F0A
:102DA0003F4F80589F4FF8E5EF0EF11C40EBE416C3
:102DB000F10409F0C2CF80E00E94E3098FE00E9495
:102DC000030C0F5F1F4F0931110509F049CFDD20BA
:102DD00011F02F9A2D9880E991E00E94540B2D9AC2
:102DE00047CF9091A90380914101A92FA81B8A2F59
:102DF00020910001A21748F48F5F821708F076CF68
:102E000081E083BF889513BE71CF81E0809340013C
:102E100090934101EEE3F1E08081918101968083FE
:102E2000918380E20E940E0C898380E40E940E0C44
:102E30008A8380E80E940E0C8B8380E10E940E0C36
:102E40008C8388E00E940E0C8D8384E00E940E0C1F
:102E50008E83BE016F5F7F4F2BE933E0A1EAB3E0C1
:102E6000FB019191BF01992319F081E04C9141112F
:102E700080E0F90181939F019D9325964EAD5FAD52
:102E800025976417750761F70091020110910301FE
:102E90000230110508F0DEC1F801E25EFE4F8081CC
:102EA000882309F463C08091A103882349F08091AD
:102EB000990390919A03089790939A0380939903AA
:102EC0008091A203882349F08091990390919A03FD
:102ED000089690939A03809399038091A303882383
:102EE00049F08091970390919803089790939803E5
:102EF000809397038091A403882349F080919703DE
:102F000090919803089690939803809397038091EB
:102F1000990390919A0397FF04C010929A0310921C
:102F200099038091990390919A038F3F910539F00D
:102F300034F08FEF90E090939A03809399038091FF
:102F400097039091980397FF04C0109298031092F2
:102F500097038091970390919803803F910534F0F7
:102F60008FEE90E0909398038093970385E4809F81
:102F7000F001819FF00D1124E35FFC4F80818111EE
:102F80000AC081E080830230110528F470E060E01F
:102F9000C8010E94EF1185E4809FF001819FF00D30
:102FA0001124E35FFC4F16821582D12CC12C5F01E6
:102FB000BF016D5F7F4F63967FAF6EAF6397CF01A9
:102FC000059629969FAF8EAF2997D801A45EBE4F74
:102FD000A196BFAFAEAFA1976396EEADFFAD63977D
:102FE0000190F081E02D2F96FFAFEEAF2F97CE1618
:102FF000DF060CF036C22996AEADBFAD29978D9194
:103000009C9148970CF02DC2A196EEADFFADA19713
:10301000E080F12C97012C0D3D1DF4E1F29FC001E1
:10302000F39F900D11249C012F5C3D4F3901490104
:1030300034E0830E911CF30184819581A681B781D0
:1030400080879187A287B387FFEFCF1ADF0AD3016A
:1030500053968C91882309F4BFCFB301C8010E9415
:103060007D0D882309F4B8CFC6010197E80EF91E3B
:10307000B4E1BE9DC001BF9D900D1124FC01EF5C29
:10308000FD4F7F01160127967FAE6EAE2797930105
:10309000245F3F4F67963FAF2EAF67976B969FAE0B
:1030A0008EAE6B97A301425F5F4F6D965FAF4EAFE1
:1030B0006D975FEF5C0D6E965FAF6E972F966EAD5E
:1030C0007FAD2F976215730509F486CF2996AEADB3
:1030D000BFAD29978D909C90B8E18B1691040CF0B0
:1030E0007BCFF70187A1882309F4ADC0B7016C5EDF
:1030F0007F4FC8010E947D0D882309F4A4C0279644
:10310000AEADBFAD27974D905D906D907C90D7018F
:1031100054962D913D914D915C9157972D962CAFE2
:103120003DAF4EAF5FAF2D976796EEADFFAD6797A2
:1031300060817181072E000C880B990B0E940C1E78
:10314000A30192010E94631D2D962CAD3DAD4EADA5
:103150005FAD2D970E94BC1E18160CF074C0D701ED
:1031600090966D917C91072E000C880B990B0E9414
:103170000C1E2D962CAD3DAD4EAD5FAD2D970E9432
:10318000631D9B01AC01C301B2010E94CF1D87FFEB
:103190005AC06B96EEADFFAD6B9740805180628058
:1031A0007380D70158962D913D914D915C915B971D
:1031B0002D962CAF3DAF4EAF5FAF2D976D96EEAD18
:1031C000FFAD6D9760817181072E000C880B990B04
:1031D0000E940C1EA30192010E94631D2D962CAD2E
:1031E0003DAD4EAD5FAD2D970E94BC1E18165CF52F
:1031F000D70192966D917C91072E000C880B990B4C
:103200000E940C1E2D962CAD3DAD4EAD5FAD2D97A1
:103210000E94631D9B01AC01C301B2010E94CF1D3E
:1032200087FF11C0F501E80DF91D6E96BFAD6E97D1
:10323000B58B25A6EFEF8E1A9E0A2996AEADBFADCF
:1032400029978D929C92BFEF2B1A3B0AE4E1EE0E78
:10325000F11C34CF17FF8ACE209102013091030177
:1032600037FDD1C390E0E7E1F4E091119FEF8FEFDC
:1032700091939193919391938150D0F7912C812CBC
:1032800045E4429FC001439F900D1124AC01405F73
:103290005C4F6D965FAF4EAF6D97B901645E7E4F28
:1032A000A9967FAF6EAFA9976D96AEADBFAD6D9786
:1032B0008D919C91881699060CF414C220912602D7
:1032C0003091270227963FAF2EAF2797A2E4B1E0B7
:1032D000F12CE12CF7E09F2E27966EAD7FAD27975E
:1032E000E616F7060CF08FC315964C911597141639
:1032F0000CF041E013968D919C91149797FD0396E5
:1033000095958795959587959C012E5F3F4F2996BA
:103310003FAF2EAF299711968D919C91129797FDF3
:1033200003969595879595958795809656E04502E5
:10333000900111242E5F3F4FB901759567957595E2
:1033400067952F967FAF6EAF2F971D0176E0270E02
:10335000311C442E440F5508F10121911F012223F5
:1033600009F44CC330EE320F3F3508F02FE3205202
:10337000330B929EA001939E500D11249A01235A63
:103380003F4E2B963FAF2EAF2B97D12CC12C70E028
:1033900060E02B96EEADFFAD2B97E60FF71F649024
:1033A000A601559547955595479529962EAD3FAD64
:1033B0002997420F531F9A0113E0359527951A95C7
:1033C000E1F7F901F695FE2FEE27F795E79563965D
:1033D000FFAFEEAF63979A01277033278824839459
:1033E00001C0880C2A95EAF7B12CA12C04E010E06A
:1033F000712C9301002E02C0359527950A94E2F7AF
:1034000020FF19C095013595279535952795280FEB
:10341000391F2038310578F44034510560F4639643
:10342000EEADFFAD63972E0F3F1FF901E95EFB4F35
:1034300020812829208301501109A40CB51C0F3FBD
:103440001007B9F66F5F7F4FC40CD51C673071054C
:1034500009F09FCF2F962EAD3FAD2F97820F931F70
:103460007BCF85E4809FF001819FF00D1124E35F05
:10347000FC4FA388B4887F01D12CC12C992493944C
:10348000CA14DB04BCF5D70118964D905D906D9081
:103490007C901B9720E030E0A901C301B2010E949B
:1034A000BC1E1816B4F429E838E848E85CE3C30108
:1034B000B2010E94621D2B013C0120E030E0A90115
:1034C0000E94CF1D181664F4F7014086518662866B
:1034D0007386BFEFCB1ADB0AE6E0EE0EF11CD0CF0D
:1034E000D70118961D921D921D921C921B971C9637
:1034F0009C92EFCF0230110528F461E070E0C80122
:103500000E94EF11B12CA12C25E4209FC001219F26
:10351000900D11249C01205F3C4F7901A801445E6D
:103520005E4F6A01A4E19A2ED7012D913C91A2161B
:10353000B3060CF04BC0F60180818A0D9B2D911DC6
:10354000989EF001999EF00D1124EF5CFD4F838948
:10355000882341F1209102013091030182892115D4
:10356000310529F02130310531F060E009C08823B0
:10357000E1F361E005C08823C1F369E08130C9F758
:1035800070E02115310531F02130310579F090E0FE
:1035900080E004C0811114C081E093E141E050E07B
:1035A0000E94940DFFEFAF1ABF0ABECF882329F007
:1035B000813049F080E093E1F1CF8FEF92E1EECFDF
:1035C00082E093E1EBCF86EF92E1E8CF8091300289
:1035D000882309F473C08091010187FD6FC0082E14
:1035E000000C990B821793070CF068C0F801E45E99
:1035F000FE4F2081820F911D44E1489F9001499F19
:10360000300D1124A9014F5C5D4F7A01DA01539608
:103610008C915397882309F451C080902C0290908C
:103620002D02A0902E02B0902F02A50194016D9161
:103630007D918D919C910E94621D20E030E040E0E0
:1036400053E40E94621D2DEC3CEC4CEC5DE30E94C7
:10365000C11EA50194010E94631D60932C0270930A
:103660002D0280932E0290932F028090280290903A
:103670002902A0902A02B0902B02A5019401F70123
:1036800064817581868197810E94621D20E030E00F
:1036900040EF52E40E94621D2DEC3CEC4CEC5DE3EB
:1036A0000E94C11EA50194010E94631D609328021F
:1036B0007093290280932A0290932B0285E4809FC5
:1036C000F001819FF00D1124E35FFC4F8389948901
:1036D000181619060CF0C0CD1486019709F4BCCD5C
:1036E000128ABACDA996AEADBFADA9978C91880DBF
:1036F000992D911DE4E1E89FD001E99FB00D1124BF
:10370000AF5CBD4F53968C915397882309F472C1D7
:1037100050968C915097282F082E000C330B253093
:10372000310508F067C1FBE08F02C0011124FC01E4
:10373000E65DFF4E459154916F965FAF4EAF6F9728
:10374000FC01E45DFF4E65917491A1967FAF6EAF71
:10375000A197FC01E25DFF4E4491FC01E15DFF4E4B
:1037600085919491A3969FAF8EAFA397220F331F9D
:10377000F901EE5EFE4FC080D180C114D10409F47E
:1037800039C114966D917D918D919C911797619699
:103790006CAF7DAF8EAF9FAF619760912802709143
:1037A000290280912A0290912B022D966CAF7DAF59
:1037B0008EAF9FAF2D976D917D918D919C91659668
:1037C0006CAF7DAF8EAF9FAF659780912C029091CB
:1037D0002D02A0912E02B0912F0269968CAF9DAF61
:1037E000AEAFBFAF69972396AEADBFAD2397E0E410
:1037F0001D92EA95E9F7712C612C242F30E0A796F1
:103800003FAF2EAFA797A1964EAD5FADA1976416BF
:1038100075060CF0EFC02D962CAD3DAD4EAD5FADF5
:103820002D9761966CAD7DAD8EAD9FAD61970E9479
:10383000621D20E030E040E85EE30E94C11E0E946D
:10384000D41D6E5F7F4FCB01860D971D29969FAFCC
:103850008EAF299763E0959587956A95E1F7DC012E
:10386000B695BA2FAA27B795A7956B96BFAFAEAFFF
:103870006B9729968EAD9FAD299787709927222443
:10388000239401C0220C8A95EAF7FE0131962F019C
:10389000312C27961FAE1EAE279710E000E0C20124
:1038A00023962EAD3FAD2397821B930BA7964EAD6B
:1038B0005FADA797841795070CF098C00115110507
:1038C00009F474C0D2018C91382A01501109760193
:1038D000D2013D922D012796AEACBFAC2797D12CDB
:1038E000C12CE32DF0E0A596FFAFEEAFA5976F9644
:1038F0002EAD3FAD6F97A216B3060CF04BC080E81B
:1039000090E00C2C02C0959587950A94E2F7A59655
:103910004EAD5FADA59784239523892B81F16996E0
:103920002CAD3DAD4EAD5FAD699765966CAD7DAD8F
:103930008EAD9FAD65970E94621D20E030E040E8AB
:103940005EE30E94C11E0E94D41D605E7F4F6A0D1F
:103950007B1D6038710598F429968EAD9FAD29972F
:103960008034910560F46B96AEADBFAD6B976A0F76
:103970007B1FFB01E95EFB4F808182298083BFEFC3
:10398000CB1ADB0AEFEFAE1ABE0AF8E0CF16D1046D
:1039900009F0ADCF27962EAD3FAD2797285F3F4F5B
:1039A00027963FAF2EAF2797670179CF7601BFEFFC
:1039B000EB1AFB0AA396EEADFFADA3971E161F06EA
:1039C00094F4F6018491D2019C91392A811109C0A5
:1039D000F70104917601F2E0EF0EF11C0150110B9A
:1039E00077CF382675CFF601349072CF3FEF631A48
:1039F000730A09CF4FEF841A940A56CC3FEFE31AAB
:103A0000F30A969669CC80E00E94E3096FC9F999A0
:103A1000FECF92BD81BDF89A992780B50895262FD3
:103A2000F999FECF92BD81BDF89A019700B40216B4
:103A300039F01FBA20BD0FB6F894FA9AF99A0FBE62
:103A40000895052E97FB1EF400940E94381D57FD23
:103A500007D00E94401D07FC03D04EF40C94381D83
:103A600050954095309521953F4F4F4F5F4F0895AA
:103A700090958095709561957F4F8F4F9F4F0895DA
:103A8000A1E21A2EAA1BBB1BFD010DC0AA1FBB1F62
:103A9000EE1FFF1FA217B307E407F50720F0A21BD4
:103AA000B30BE40BF50B661F771F881F991F1A9441
:103AB00069F760957095809590959B01AC01BD016B
:103AC000CF0108955058BB27AA270E947A1D0C9455
:103AD000821E0E94741E38F00E947B1E20F039F472
:103AE0009F3F19F426F40C94711E0EF4E095E7FB49
:103AF0000C946B1EE92F0E94931E58F3BA176207AD
:103B000073078407950720F079F4A6F50C94B51E89
:103B10000EF4E0950B2EBA2FA02D0B01B9019001E8
:103B20000C01CA01A0011124FF27591B99F0593F2C
:103B300050F4503E68F11A16F040A22F232F342F74
:103B40004427585FF3CF469537952795A795F040C2
:103B50005395C9F77EF41F16BA0B620B730B840BD7
:103B6000BAF09150A1F0FF0FBB1F661F771F881F8F
:103B7000C2F70EC0BA0F621F731F841F48F48795E7
:103B800077956795B795F7959E3F08F0B0CF9395D9
:103B9000880F08F09927EE0F9795879508950E9452
:103BA000471E08F481E008950E94DB1D6894B1115E
:103BB0000C94B61E08950E949B1E88F09F5798F0A3
:103BC000B92F9927B751B0F0E1F0660F771F881F22
:103BD000991F1AF0BA95C9F714C0B13091F00E943C
:103BE000B51EB1E008950C94B51E672F782F882775
:103BF000B85F39F0B93FCCF3869577956795B39563
:103C0000D9F73EF490958095709561957F4F8F4FD1
:103C10009F4F0895E89409C097FB3EF490958095D6
:103C2000709561957F4F8F4F9F4F9923A9F0F92F82
:103C300096E9BB279395F695879577956795B79500
:103C4000F111F8CFFAF4BB0F11F460FF1BC06F5FE6
:103C50007F4F8F4F9F4F16C0882311F096E911C0F8
:103C6000772321F09EE8872F762F05C0662371F019
:103C700096E8862F70E060E02AF09A95660F771F2D
:103C8000881FDAF7880F9695879597F90895990F09
:103C90000008550FAA0BE0E8FEEF16161706E80716
:103CA000F907C0F012161306E407F50798F0621B37
:103CB000730B840B950B39F40A2661F0232B242B0C
:103CC000252B21F408950A2609F4A140A6958FEF2B
:103CD000811D811D089597F99F6780E870E060E07D
:103CE00008959FEF80EC089500240A941616170695
:103CF00018060906089500240A94121613061406DD
:103D000005060895092E0394000C11F4882352F03F
:103D1000BB0F40F4BF2B11F460FF04C06F5F7F4FF7
:103D20008F4F9F4F089557FD9058440F551F59F0DE
:103D30005F3F71F04795880F97FB991F61F09F3F98
:103D400079F087950895121613061406551FF2CFC1
:103D50004695F1DF08C0161617061806991FF1CF11
:103D600086957105610508940895E894BB27662738
:103D70007727CB0197F908950E94471E08F48FEF2B
:103D800008950E94D41E0C94821E0E94741E38F066
:103D90000E947B1E20F0952311F00C946B1E0C9456
:103DA000711E11240C94B61E0E94931E70F3959FF1
:103DB000C1F3950F50E0551F629FF001729FBB2722
:103DC000F00DB11D639FAA27F00DB11DAA1F649FBE
:103DD0006627B00DA11D661F829F2227B00DA11D71
:103DE000621F739FB00DA11D621F839FA00D611DF7
:103DF000221F749F3327A00D611D231F849F600D18
:103E0000211D822F762F6A2F11249F5750409AF040
:103E1000F1F088234AF0EE0FFF1FBB1F661F771FCC
:103E2000881F91505040A9F79E3F510580F00C9497
:103E30006B1E0C94B61E5F3FE4F3983ED4F3869558
:103E400077956795B795F795E7959F5FC1F7FE2B37
:103E5000880F911D9695879597F90895EE0FFF1F8E
:103E60000590F491E02D0994FB01DC014150504094
:103E700048F001900D920020C9F701C01D924150F9
:0A3E80005040E0F70895F894FFCFDA
:103E8A0010FFFFFFFFFFFFFF00E10000000000003E
:103E9A0005069302CA00C000B600AC000005000087
:103EAA0000C1808100000000000000410A680B6226
:0A3EBA000A570AA80A660A840A00E3
:00000001FF
